S025000062696E2F64656D6F70726F675F6F6C696D65785F65666D3332673838302E737265634A
S11320006801002099220000E5260000E526000072
S1132010E5260000E5260000E5260000E526000090
S1132020E5260000E5260000E5260000E526000080
S1132030E5260000E5260000E5260000D126000084
S1132040E5260000E5260000E5260000E526000060
S1132050E5260000E5260000E5260000E526000050
S1132060E5260000E5260000E5260000E526000040
S1132070E5260000E5260000E5260000E526000030
S1132080E5260000E5260000E5260000E526000020
S1132090E5260000E5260000E5260000E526000010
S11320A0E5260000E5260000E5260000B52800002E
S11320B0E5260000E5260000EE11AA5510B50446F9
S11320C04FF48843C4F20803DB6A13F0040F0CD006
S11320D04FF48840C4F2080043F20943C0F20003FD
S11320E0984720704FF0010010BD4FF0000010BD64
S11320F070B584B043F23C43C0F200036E460FCB8C
S113210086E80F004FF44240C0F202004FF0010194
S113211042F62954C0F20004A0474FF002004FF0E9
S113212006014FF004024FF0010343F21525C0F2FB
S11321300005A8474FF002004FF007014FF00102DD
S11321404FF00003A8474FF40C50C0F204004FF0C6
S11321500101A0474FF00300C0F212004FF002014A
S113216043F2B903C0F2000398474FF4AA55C0F2F2
S1132170160528464FF0010142F67933C0F20003F8
S1132180984728464FF00101A0474FF000058DF80D
S113219000504FF48844C4F208042046694643F2D0
S11321A0A933C0F200039847204629464FF416523B
S11321B043F20933C0F2000398474FF00303636509
S11321C04FF00403636320464FF0050143F26D337F
S11321D0C0F20003984704B070BD00BF08B540F2D8
S11321E00903C2F200031B78CBB940F20C00C2F21F
S11321F0000042F2BD03C0F200039847012848D111
S113220040F20903C2F200034FF001021A7040F2D7
S11322100803C2F200034FF000021A7008BD40F236
S11322200803C2F2000318781A4BC01842F2BD0327
S1132230C0F20003984701282BD140F20803C2F2F0
S113224000031A7802F10102D2B21A7040F20C03B0
S1132250C2F200031B7893421BD140F20903C2F27D
S113226000034FF000021A7040F20C03C2F20003A4
S11322705B78FF2B0DD140F20C03C2F200039B7874
S11322803BB942F24D63C0F2000398474FF0B903E3
S1132290984708BD0D00002008B516498D4640F248
S11322A00002C2F2000240F20803C2F200039A42A2
S11322B011D243F24C42C0F2000240F20003C2F2D7
S11322C0000340F20800C2F2000052F8041B43F875
S11322D0041B8342F9D3084808494FF0000288429E
S11322E0B8BF40F8042BFADB42F29D33C0F200037E
S11322F0984708BD680100200800002068000020FD
S113230062B6704708B54FF42040C4F2080042F6A4
S11323109913C0F20003984708BD00BF10B542F2FC
S1132320C563C0F200039847044640F25003C2F26A
S113233000031B68C31AB3F5FA7F2ED340F254038B
S1132340C2F200031B7893B940F25403C2F20003B3
S11323504FF001021A704FF42040C4F208004FF00D
S1132360000142F6F103C0F20003984710E040F286
S11323705403C2F200034FF000021A704FF42040DD
S1132380C4F20800114642F6F103C0F20003984774
S113239040F25003C2F200031C6010BD30B583B09C
S11323A042F2CD73C0F20003984748F2FC13C0F622
S11323B0E0731B681B0E14D14AF20C03C4F20C0325
S11323C01A6822F070021A6046F22003C4F20C0369
S11323D01A6822F060421A601A6862F060621A6039
S11323E001E0032B22D846F22003C4F20C031A683E
S11323F022F4FC521A6048F24002C4F20C024FF07C
S11324000003136048F24402C4F20C02136048F261
S11324105802C4F20C02136048F26002C4F20C02C7
S1132420136048F27802C4F20C02136001A843F26C
S11324301943C0F2000398479DF80430012B17D1CB
S11324409DF805303BB948F24003C4F20C031A6806
S113245042F002021A609DF80530012B9FBF48F23A
S11324604403C4F20C031A6842F0010298BF1A60D4
S113247048F2F013C0F6E0731A684BF6FF13C4F683
S11324808A439A4230D848F24403C4F20C031A68CF
S113249042F490421A6048F2B412C0F6E072116835
S11324A001F4FE4110681568146804F07F0405F413
S11324B0FE4244EA020200F07F0042EA004242EA9D
S11324C0014142F23402C4F20002116048F2C8121F
S11324D0C0F6E072116844F22C02C4F200021160EA
S11324E01A6822F490421A604FF000004FF0010184
S11324F00A4643F24503C0F2000398474FF40043F1
S1132500C4F20C031A6C42F00F021A645A6C6FEA9C
S113251012426FEA02425A644FF44070C0F204005F
S11325204FF0000142F62954C0F20004A0474FF4D2
S11325309850C0F204004FF00001A0474FF44C50F3
S1132540C0F204004FF00001A0474FF42240C0F253
S113255002004FF00001A0474FF40070C0F20200E7
S11325604FF00001A0474FF49050C0F202004FF02A
S11325700001A0474FF40850C0F202004FF00001E0
S1132580A0474FF44850C0F202004FF00001A047AA
S11325904FF4E440C0F202004FF00001A0474FF4B2
S11325A00240C0F202004FF00001A0474FF4324055
S11325B0C0F202004FF00001A0474FF46240C0F2A5
S11325C002004FF00001A0474FF47240C0F2020035
S11325D04FF00001A0474FF45240C0F202004FF008
S11325E00001A0474FF001004FF009014FF0050230
S11325F0034643F21524C0F20004A0474FF0010043
S11326004FF0020143F2F513C0F20003984742F27F
S11326100533C0F20003984742F26963C0F2000335
S1132620984742F20133C0F20003984742F2F103A3
S1132630C0F20003984742F21D35C0F2000542F291
S1132640DD14C0F20004A847A047FCE74EF21003D3
S1132650CEF200034FF000021A60704740F25803B4
S1132660C2F200031860704708B54FF02000C0F2B2
S1132670040042F65D63C0F20003984744F6D35366
S1132680C1F26203A3FB00204FEA901000F1FF3077
S11326904EF21003CEF2000358604FF46D42CEF2B6
S11326A000024FF0E00182F823104FF00000986020
S11326B04FF007021A6042F25D63C0F200039847CC
S11326C008BD00BF40F25803C2F200031868704707
S11326D040F25803C2F200031A6802F101021A60C0
S11326E0704700BFFEE700BF4FF40043C4F20C0381
S11326F0DB6A03F47053B3F5805F48D0B3F5005F31
S113270003D0B3F5006F0CD105E040F20003C2F230
S113271000031868704740F20403C2F2000318680B
S113272070474FF40043C4F20C03DB6803F4E06326
S1132730B3F5007F19D004D80BB3B3F5807F23D150
S113274018E0B3F5806F25D0B3F5A06F03D0B3F5CF
S1132750407F19D104E04FF47C50C0F2AB107047B5
S113276049F68070C0F2D50070474DF6C000C0F243
S1132770A70070474CF6C070C0F26A00704744F27C
S11327804020C0F20F0070474FF0000070474FF434
S11327900040704746F64070C0F24010704700BFDA
S11327A008B542F2E963C0F2000398474FF40043CE
S11327B0C4F20C035B6803F00F0320FA03F040F249
S11327C06402C2F20002106008BD00BF704700BF7F
S11327D04FF40040704700BF40F20003C2F2000310
S11327E0186870471F2AC4BF203A04314FF0010310
S11327F003FA02F2072924D8DFE801F004080C10D8
S113280014181C20036C1A4302647047436C1A4367
S113281042647047836C1A4382647047C36C1A43E2
S1132820C2647047036D1A4302657047436D1A43CF
S113283042657047836D1A4382657047C36D1A43BE
S1132840C26570471F2AC4BF203A04314FF0010308
S113285003FA02F207292CD8DFE801F004090E1369
S1132860181D2227036C23EA020202647047436C9A
S113287023EA020242647047836C23EA0202826400
S11328807047C36C23EA0202C2647047036D23EAF3
S1132890020202657047436D23EA020242657047F3
S11328A0836D23EA020282657047C36D23EA020244
S11328B0C26570474FF42043C4F208034FF0FF325F
S11328C05A6240F25C03C2F200031A6802F1010288
S11328D01A6070474FF00003036403654364436563
S11328E083648365C364C365436E002BFCD1704766
S11328F038B50B293FD8DFE801F03A060B0F14195D
S11329001E23282D31354FF003034FF0010432E02C
S11329104FF003031C462EE04FF003034FF0000476
S113292029E04FF003034FF0020424E04FF02703A3
S11329304FF000041FE04FF027034FF003041AE0A8
S11329404FF001034FF0030415E04FF001034FF083
S1132950020410E04FF001031C460CE04FF00103A9
S11329601C4608E04FF007034FF0030403E04FF068
S11329700F034FF003043AB121461A4642F2E573BD
S1132980C0F20003984738BD21461A4642F6450373
S1132990C0F20003984738BD10B504464FF4004315
S11329A0C4F20C039A6A22F003029A629A6A42F011
S11329B002029A629A6D42F004029A659A6E22F4B7
S11329C040729A669A6E42F440729A664FF000031F
S11329D08362636E002BFCD14FF0FF3363624FF4CC
S11329E06143CEF200034FF000621A604FF001031E
S11329F0A36241F60B7363604FF40043C4F20C030B
S1132A004FF00002DA67204642F6D503C0F2000315
S1132A10984740F2FF33A3604FF005032360636ED1
S1132A20002BFCD14FF48073C0F21C03E360636E8F
S1132A30002BFCD14FF001036362A36210BD00BF01
S1132A4000F1047001EBC0004FEA8000026070479F
S1132A504FF00003C4F20C035B6803F00702032A7F
S1132A600CD8DFE802F00202070723F0070343F063
S1132A70010303E023F0070343F003034FF00002D4
S1132A80C4F20C0253607047B0FA80F0C0B2C0F1D7
S1132A901F0070474FF00003C4F20C035B684DF64F
S1132AA0FF32CFF60B72821842F2FF31C0F2F4010A
S1132AB08A420BD803F00702A2F10202012A23F092
S1132AC0070394BF43F0030343F001034FF4105290
S1132AD0C0F2F402904209D803F00702A2F1020204
S1132AE0012A23F0070398BF43F002034FF00002CA
S1132AF0C4F20C025360704749F68070C0F2D500EE
S1132B00704700BF4FF40043C4F20C035B6D13F035
S1132B10010F06D14FF40042C4F20C02136D1842A7
S1132B20FCD1704708B54FF40043C4F20C039B6A10
S1132B304FEA400023FA00F303F00303022B09D009
S1132B40032B0DD0012B13D142F2D173C0F2000339
S1132B50984708BD42F2D973C0F20003984708BDF4
S1132B6042F2A173C0F2000398474FEA500008BD37
S1132B704FF0000008BD00BF10B50C46C0F30313AE
S1132B8003F1FF33032B00F2CE80DFE803F00213DE
S1132B903390084642F68923C0F2000398474FF465
S1132BA00043C4F20C039A6822F00F0240EA0202C6
S1132BB09A6010BD42F65123C0F2000398472046A4
S1132BC042F68923C0F2000398474FF40043C4F24D
S1132BD00C035A6822F00F0240EA02025A6042F2E1
S1132BE0A173C0F20003984742F69523C0F2000394
S1132BF0984710BD41F23043C0F20A03984224D0F2
S1132C004FF03003C0F20C03984236D04FF4866381
S1132C10C0F20803984240F086804FF0040042F668
S1132C200533C0F200039847204642F68923C0F2D8
S1132C30000398474FF40043C4F20C039A6E22F049
S1132C400F0240EA02029A6610BD4FF0040042F6F9
S1132C500533C0F200039847204642F68923C0F2A8
S1132C60000398474FF40043C4F20C039A6E22F019
S1132C70F00242EA00129A6610BD4FF0040042F6D8
S1132C800533C0F200039847204642F68923C0F278
S1132C90000398474FF40043C4F20C039A6EA0F16A
S1132CA0100022F4407242EA00229A6610BD4FF4EA
S1132CB0A863C0F21403984206D04FF4AA53C0F29A
S1132CC0160398422FD117E04FF0400042F6053327
S1132CD0C0F200039847204642F68923C0F200035D
S1132CE098474FF40043C4F20C031A6F22F0030216
S1132CF040EA02021A6710BD4FF0400042F6053365
S1132D00C0F200039847204642F68923C0F200032C
S1132D1098474FF40043C4F20C031A6F22F03002B8
S1132D2042EA00121A6710BD70B50D46C0F30323C2
S1132D3003F1FF33052B3AD8DFE803F0082D3217EF
S1132D401E0348F27804C4F20C042DE0C0F30436E8
S1132D5048F20804C4F20C04204631462A4642F6DE
S1132D604123C0F20003984770BD4FF0010348F2BD
S1132D705804C4F20C0405E04FF0100348F2600458
S1132D80C4F20C04C0F30436184642F60533C0F20C
S1132D9000039847E0E748F24404C4F20C0403E05B
S1132DA048F24004C4F20C04C0F30436D4E770BD06
S1132DB000F00F0000F1FF30032842D8DFE800F0F4
S1132DC0051B2E024FF0070070474FF40043C4F276
S1132DD00C03D86A00F47050B0F5805F34D0B0F5BD
S1132DE0005F05D0B0F5006F0CBF042005207047CC
S1132DF04FF0020070474FF40043C4F20C03986A8A
S1132E0000F00300022822D0032804D001280CBFBC
S1132E100320012070474FF0060070474FF4004331
S1132E20C4F20C03986A00F00C00022812D00328A4
S1132E3004D001280CBF0320012070474FF0060086
S1132E4070474FF0000070474FF0030070474FF099
S1132E50020070474FF00200704700BF08B500F44D
S1132E607810B0F5402F74D014D8B0F5802F40D02E
S1132E7005D848B3B0F5003F40F0E0802AE0B0F553
S1132E80002F44D0B0F5202F52D0B0F5C02F40F021
S1132E90D58034E0B0F5A01F00F08C8007D8B0F5E1
S1132EA0602F67D0B0F5901F40F0C8807AE0B0F58D
S1132EB0C01F00F0A180B0F5D01F00F0B980B0F5BC
S1132EC0B01F40F0BB8086E042F2E963C0F2000329
S1132ED0984708BD42F2E963C0F2000398474FF4F3
S1132EE00043C4F20C039B6803F00F0320FA03F0C1
S1132EF008BD42F2A173C0F20003984708BD4FF029
S1132F00000042F62533C0F20003984708BD4FF095
S1132F10000042F62533C0F2000398474FF4004303
S1132F20C4F20C039B6E03F00F0320FA03F008BDF8
S1132F304FF0000042F62533C0F2000398474FF4E7
S1132F400043C4F20C039B6EC3F3031320FA03F093
S1132F5008BD4FF0000042F62533C0F20003984745
S1132F604FF40043C4F20C039B6EC3F3012320FA15
S1132F7003F008BD4FF0000042F62533C0F2000311
S1132F8098474FF40043C4F20C039A6EC2F3012233
S1132F9020FA02F0DB6F03F0070303F10103B0FB37
S1132FA0F3F008BD4FF0010042F62533C0F20003F0
S1132FB0984708BD4FF0010042F62533C0F20003E4
S1132FC098474FF40043C4F20C031B6F03F0030350
S1132FD020FA03F008BD4FF0010042F62533C0F299
S1132FE0000398474FF40043C4F20C031B6FC3F370
S1132FF0011320FA03F008BD4FF00400C0F21800DA
S113300042F6B153C0F200039847072807D00828B6
S11330100BD142F2E963C0F20003984708BD42F6BF
S1133020F923C0F20003984708BD4FF0000008BD23
S113303042F6F923C0F20003984708BD4FF00000A0
S113304008BD00BF10B5042835D8DFE800F0120D24
S1133050170308004FF001044FF0020012E04FF094
S113306010044FF020000DE04FF040044FF08000BA
S113307008E04FF480744FF4007003E04FF0040450
S11330804FF0080069B14FF40043C4F20C031C6212
S113309062B14FF40042C4F20C02D36A1842FCD06D
S11330A004E04FF40043C4F20C03186243F2DD134E
S11330B0C0F20003984710BD10B500F00F000128BE
S11330C006D0002800F08880032800F285803BE0C9
S11330D0A1F1020103297FD8DFE801F00210070BF8
S11330E04FF000004FF004040CE04FF002000446DF
S11330F008E04FF003004FF0010403E04FF001003B
S11331004FF003044FF001010A4643F24503C0F2B5
S11331100003984742F65123C0F2000398474FF446
S11331200043C4F20C035C6243F2DD13C0F20003FB
S1133130984742F2A173C0F20003984742F69523E0
S1133140C0F20003984710BD022814BF02240024D3
S113315001F1FF3105293FD8DFE801F02C03103ECF
S11331603E1C4FF000004FF001010A4643F24503B4
S1133170C0F2000398474FF002021DE04FF0010037
S11331800146024643F24503C0F2000398474FF05C
S1133190010211E048F24000C4F20C004FF00201B9
S11331A04FF0010242F64123C0F2000398474FF06A
S11331B0030201E04FF000024FF40043C4F20C0399
S11331C0996A02FA04F24FF0030000FA04F421EAC7
S11331D0040442EA04049C6210BD00BF4FF400439F
S11331E0C4F20C03DA6A40F26003C2F200031A80EC
S11331F0704700BF4FF4C043C4F2000300EBC000AB
S113320053F8202022F0030241EA020243F820206E
S1133210704700BFF0B41446E2B16BB14FF0010542
S113322005FA01F500EBC0024FEA820202F1804286
S113323002F5C04215610DE04FF0010505FA01F5F4
S113324000EBC0064FEA860646F21002C4F2000202
S1133250B2185560072916D800EBC0024FEA820263
S113326002F1804202F5C04257684FEA81054FF0EF
S11332700F0606FA05F627EA060604FA05F546EAF5
S11332800505556017E000EBC0024FEA820202F127
S1133290804202F5C04297684FEA8105A5F12005F6
S11332A04FF00F0606FA05F627EA060604FA05F5B6
S11332B046EA05059560E4B96BB14FF0010303FAE2
S11332C001F100EBC0004FEA800000F1804000F5FE
S11332D0C04001610DE04FF0010303FA01F100EB7E
S11332E0C0004FEA800046F21003C4F20003C31882
S11332F05960F0BC704700BF036C13F0010F02D19A
S1133300436C1942FCD1704738B50446154608464B
S1133310D1B94FF48043C4F208039C420BD04FF45C
S11333208843C4F208039C4204BF4FF4AA50C0F27D
S113333016001AD103E04FF4A860C0F2140042F65C
S11333405D63C0F2000398474FEA4010B0FBF5F507
S1133350A5F120054FEAC50520464FF0040143F2CC
S1133360F923C0F200039847E56038BD38B5044638
S11333706FEA010505F0050541EA45054FF0020134
S113338043F2F923C0F200039847656038BD00BFDB
S113339031B1436C002BFCD14FF00103036470473F
S11333A04FF000030364704770B504460D464FF0B8
S11333B0020143F2F923C0F2000398474FF00A03D5
S11333C0636020464FF0010143F29136C0F20006DB
S11333D0B04723682A7B23F01C0342EA03036A7B79
S11333E01343AA7B1343236020466968AA6843F207
S11333F00933C0F2000398472B78636020464FF0EE
S11334000001B04770BD00BF836813F0200FFBD0EC
S1133410C069C0B2704700BF4FF6D073CEF20F033D
S11334201A6902F03F0202709A6902F0F002DB6945
S1133430C3F3031342EA030343707047050000001B
S10F3440000000008025000000000000D7
S10B344C008000000048E801C3
S9032000DC
